:080000007522001200EF01332C
:20000B00C2A9C28CDF013230BC08758C51758A00012E201208758CF9758A00012E758CFF34
:20002B00758A40D28CD2A932E47821F6D8FD758108120FD9D2AF12004B12011E01330141A6
:20004B00C210C212C2BC7B0275260012007FF52704F9782B12007FF6082526F526D9F51237
:20006B00007FB526067455120092227401120092DBD60133900000209808A3AC83BCFFF7B4
:20008B000133E599C298223099FDC299F599227B02752600782BAE27E527141200927F146F
:2000AB00DFFEE6081200927F14DFFE2526F526DEF1E5261200927F14DFFE12007FB4550167
:2000CB0022DBCE0133752B5575270112009A22752B0101D33099FDC299D299201A1E201924
:2000EB001320180875CBFF75CAB8210D75CBFF75CAF4210D75CBFF75CAFA210D75CBFF7544
:20010B00CAFD75870075984075890175C834D2CAD29C22852B25852C18852D1B852D238563
:20012B002E1A852F1985301E85311D85321CC211E52530E602D211C2E6F525E518543F906C
:20014B0014CC93FDE51854C07002D2BC30E704D212C2BCE518543FB40E06D2BA740A217E95
:20016B00B42104D211217EB43504D211217EB42202D211FAE525540FB40003C21022B40128
:20018B0003020207B40205D210020785B40305D213020207B4040201DFB40503020309B457
:2001AB000605D214020207B40705D217020207B40803020C0DB40903021782B40A03021676
:2001CB0038B40B0302166AB40C0302165FB40D030201E0013375F68775F65975BF03758899
:2001EB000075B80075A8827EF07FFF8E8A8F8C7F00758901758810758701222212085F754F
:20020B0026007B0212107312106912085F9012B0021262D2814137752100D2A0D284D2A430
:20022B00C2A4C28412085FD28041372230170302028D12084B12083C2014351200922526B4
:20024B00F5261210123010E4201432E52612009212007FB4550CC214531FFB121008120FD7
:20026B00D922852D1B852E1A852F19DBBF020033B4FF0512101280CD1200DA80D91200D0E2
:20028B0080D4C21775210012084B1210879013F4021262D28274041208860202ECBA0F024E
:2002AB0080030202B3201D2BBA240280030202BE201D20BA250280030202C90202DEBA1131
:2002CB000280030202D4201F0AD28374081208860202EC201CF3D28574201208860202EC62
:2002EB002212083CF526120092E52612009212007F12088422740041EF41EF0205A1120826
:20030B005F90131C021262120395120389D282740512088602032F120395120389D2827445
:20032B000C120886C2847F64120CBAD2840205A1120395120389D283D280D284C2A47409DF
:20034B00120886C2A07F64120CBAD2A0D2A40205A1120395120389D284D283740912088635
:20036B0002037D120395120389D284D2837418120886C2A47F64120CBAD2A40205A1E51F8E
:20038B0054E54402F51F12100A2212107312106912085F22C212BA172E121069201805C259
:2003AB00A10203B1D2A1D2B4C280D280121DAA75F040D212121CD7C2D9C280D28030B4FDD7
:2003CB00D2D9C2120205A112107312106912085FBA0A02800302046DBA1E02800302041221
:2003EB00D2BCD283D284D2A01210877408120886C284C2A07F01120CBAD2A0D28474001234
:20040B000886C2BC0205A1BA1D02800302043ED2BC43800E1210877404120886C283C281D5
:20042B007B28120872D281D2837400120886C2BC0205A1BA10028003020516301F121211B0
:20044B00C3121209D2BC7F28120CBAC2BC0205A11211B312112ED2BC7F28120CBAC2BC02BA
:20046B0005A1D284752110121000D2A4D2A0BA1902800302049A120AC17E301208611212A3
:20048B003D7E3012086112123D12085F0204E8BA240280030204A481C6BA25028003020465
:2004AB00AE81C6BA0F0280030203E3301F0D121087D28074011208860204DF301D16121030
:2004CB0087D28474101208861211B312112E12085F0204F91211B312112E12085FC2A4C2A9
:2004EB008412083CD284D2A430E7F20205A1C2A4C3920C12100012083CF5F0D3920C1210E3
:20050B0000D2A4E5F030E7E60205A1E51F54FD12100ABA113F301F1A741112088612084B62
:20052B007E2012086112123D7ED012086112123D80BCD392A1741112088612084B7E201290
:20054B00086112123D7ED012086112123D120880D2848089120880301F137E30120861126C
:20056B00123D000012123D12085F0204E87B147E2012086112123D000012123D7F0A120C48
:20058B00BA7EA012086112123DDBE47E0012086112123D1208841200D022C280C2D8C2D96A
:2005AB00C2B41206A375F0FFD212120605E5F060211206B21207591206A3E5F0B4FF32E5AE
:2005CB001BC4540FB40506E5F04401A1DA74A11206651206801200922526F52612101230E2
:2005EB0010F01206B2E52612009212007F120FD922E5F0440112066580D8E51BC4540F9024
:20060B00061002126306C106D006DB06ED0701071107281200D0120C8B121069C280C2D890
:20062B00C2D9C2B4E51B540F90065E93FB1206A3C212120605782BE612066508121012DBF0
:20064B00F61206B21200D0201005120C8B80CD120FD922000408102040807908339281D211
:20066B00A1120759C2A1120759D9F1D281D2A1120759C2A1227908D2A100000000A28133B6
:20068B0000000000C2A100000000D9EBC281D2A1120759C2A1D28122D281D2A1120759C22E
:2006AB0081120759C2A122C281C2A1120759D2A1120759D28122E519C3301201D333120623
:2006CB006575F0002274A0120665E51912066522E51A23540E24A054FE120665E5191206C8
:2006EB006522E51A23540E24A054FEF5F0120665E5191206652274A0120665E51A120665C2
:20070B00E51912066522E51B23540224A0F5F0120665E51A120665E51912066522E5180379
:20072B005460F5F0E525548045F0C4540E44A0F5F030E102D28030E202D2D830E302D2D930
:20074B00120665E51A120665E5191206652200000000000022E52703547FF5272222BC19BF
:20076B001885252E85182F752705851B2B851A2C85192D12009A0200332212085F20100103
:20078B0022C210EA9415603D14603A146037121073121053121069121080BA10030207D0F4
:2007AB00BA1F02E1CAEA94216015146012BA1902E1CABA3502E1CAEA941240030207D01234
:2007CB0000D0120C8B901388021262D2810207ED752100D2A0D284D2A4C2A4C284D280E1F8
:2007EB00ED22782BBA1903120AC112080B12085F12101208D527F31200D03010C502026372
:20080B007C0012084B120828500122901460021262D2905390E1D2A5D285C2A42212083CEB
:20082B00F5F0E6B5F002D322C32274038CF0A4FF22900843ED0212630CE30D5A0E4B0FD8D4
:20084B00900852ED0212630CFC0D7B0E8B0FD8E6FE0208617EFF900868ED0212630CC10D25
:20086B00380E290FD87BA07C000000DCFCDBF822E5F0020886740101867400547F301102C8
:20088B00448012126FD2A6C2A62220BC03BC1917F52E85F02F752705851B2B851A2C85198D
:2008AB002D12009A020033222222D28212085A7402120886D2837F02120CBAC2831208844A
:2008CB000C12085FC282120828502020BC17201214D28212085A7402120886120835D283D7
:2008EB00120CBAC283120884C2822212089580BAD28312085AD28274041208861217E11292
:20090B000884C283C2820C12085F120828502020BC15201212D283D28212085A740412089C
:20092B00861208351217E3120884C283C2822212089580BCC284D28312085A120880C284A8
:20094B001217D712088412085FC2830C120828501A20BC1120120ED28312085A12088012D6
:20096B0008351217D9120884C2832212089580C4C2BCD283D28412085A1208801217EB12D8
:20098B000884C283C2840C12085F120828501B201210D283D28412085A12088012083512A7
:2009AB0017ED120884C283C2842212089580C1C2BCD283D28412085A74081208861217EB20
:2009CB00120884C283C2840C12085F120828501D201212D283D28412085A7408120886121E
:2009EB0008351217ED120884C283C2842212089580BDC2BCD284D2A4D2A012085AD280C21E
:200A0B00A41208801217D7120884C2840C12085F120828501920120ED28412085A120880D5
:200A2B001208351217D9120884C2A4C2842212089580BFC2BCD284D2A412085A1208801296
:200A4B0017CD1208840C12085FC284C2A4120828501B201210D284D2A412085A12088012FD
:200A6B0008351217CF120884C284C2A42212089580C1C2BCD284D2A412085A7410120886F8
:200A8B001217CD1208840C12085FC284C2A4120828501D201212D284D2A412085A741012BD
:200AAB0008861208351217CF120884C284C2A42212089580BD22742375F018120AEB74202D
:200ACB00120AEB7422120AEB741875F004120AEB741B120AEB7419120AEB741A120AEB228A
:200AEB00120F79E5F0120F9AC2A4C28412083CD284D2A422C2BCD284D3920C121000D2A4F4
:200B0B00D2A0D280BA191A7E1012086112123D12084B12085A12123D7F28DFFEC2A4C28445
:200B2B0022BA0F4F301F0D121087D2807401120886020B4C301D0A121087D28474101208B7
:200B4B008612122912084B12085A12123D7F10DFFE12085F301D0AC2A4C3920C12100061F7
:200B6B0070C2A4C284120828400302089B740012088622D280BA1111301F04D284618CD258
:200B8B00A17411120886020B971208807E4012086112123D12085A12123DBA113212088040
:200BAB00D284301F1BC2A4C3920C12100012083CF5F0D3920C121000D2A4E5F030E7E62249
:200BCB00C2A4C28412083CD284D2A430E7F2227F14DFFE7EC012086112123D7F10DFFE1209
:200BEB00085FC2A4C2840C1208285010D284D2A41208847F08DFFEC2A4C2842212089502DC
:200C0B000AFF1210731210697E00BA0B2FD281D282C28312084B8EF0120861C281D281123C
:200C2B00085FC283C28212083CB5F051AEF00ED2821210123010DCD283020288BA0C36D26E
:200C4B00A0D283C28412084B8EF0120861BA0C02D2A1D2A0C2A0D2A012085FC283C2841259
:200C6B00083CB5F018AEF00ED2831210123010D5D284020288BA0D0280C502028802089BFD
:200C8B007B0212007F04F527FE752600782B12007FF62526F52608DEF512007FB526067431
:200CAB0055120092227401120092DBD6020033120012BF00FD22EEA2E09290A2E19291A233
:200CCB00E29292A2E392A5A2E492A4A2E59285A2E69284A2E792A322E5905407A2A592E3E3
:200CEB00A2A492E4A28592E5A28492E6A2A392E722E519A2E092B2A2E19286A2E29297A263
:200D0B00E392DAA2E492B4A2E592D9A2E692D8A2E79280E51AA2E092A0A2E192A1A2E292AF
:200D2B00A2A2E39215BA0104A215928122EEA2E09292A2E19293A2E29294A2E392B5A2E4F7
:200D4B0092B3A2E592A5A2E692A4A2E7928522A29292E0A29392E1A29492E2A2B592E3A29F
:200D6B00B392E4A2A592E5A2A492E6A28592E722E519A2E09291A2E19290A2E292B2A2E36C
:200D8B009286A2E49297A2E592DAA2E692B4A2E792D9E51AA2E09281A2E19282A2E292A3E8
:200DAB00A2E392A2A2E492D8A2E592A1A2E69215A2E79216BA1E15201F09A2159280D39202
:200DCB00A0A1E7A21592A0D39280A1E7BA0404A2169280BA0202A1E7A21592A022A2E09299
:200DEB0091A2E19290A2E292B2A2E39286A2E49297A2E592DAA2E692B4A2E792D922A2E045
:200E0B009281A2E19282A2E292A3A2E392A2A2E492D8A2E592A1A2E69280D392A022EEA2B0
:200E2B00E09294A2E19295A2E29296A2E392B6A2E492B7A2E592B5A2E692B3A2E792A52232
:200E4B00A29492E0A29592E1A29692E2A2B692E3A2B792E4A2B592E5A2B392E6A2A592E792
:200E6B0022F590EEA2E692B3A2E792B5543FF5A022E590FEE5A0A2B392E6A2B592E7CE2266
:200E8B00E519A2E09293A2E19292A2E29291A2E39290A2E492B2A2E59286A2E69297A2E70A
:200EAB0092DAE51AA2E092A2A2E19283A2E29285A2E392A3A2E492B4A2E59282A2E6928117
:200ECB00A2E792D9BA1129301F1AD284E51BA2E092D8A2E192A1A2E2920FA2E3920D121053
:200EEB0000020F77D392A1E51BA2E092D8020F77E51BA2E092D8A2E192A1A2E29215A2E393
:200F0B009216BA240BA2E6920EA2E7920B020F2BBA250280F0BA0F29301E05D280020F773B
:200F2B00301D17D284A215920FA216301C06920E12100022920D12100022A2159280020FE9
:200F4B0077BA1007A2159280020F77BA1907A2159280020F77BA0704A2169280BA0503026F
:200F6B000F77BA0903020F77A21592A02222A2E09293A2E19292A2E29291A2E39290A2E443
:200F8B0092B2A2E59286A2E69297A2E792DA22A2E092A2A2E19283A2E29285A2E392A3A256
:200FAB00E492B4A2E59282A2E69281A2E792D97400A2E092D8A2E192A1A2E39216BA0F08BE
:200FCB00301E05D280020FD7A2169280222212085F749B547BF51F12100A12088475800041
:200FEB0075900075A00075B00375D808C2BA020FFD22D29922E521440112126F22E51F1200
:20100B00126FD2A7C2A722E51CB5190DE51DB51A08E51EB51B03D21022C3E5192401F519BD
:20102B00E51A3400F51AE51B3400F51BBA1B0674061219B72230BA03021052BA0A09201F69
:20104B0006D2DA0000C2DA22E5255480700AE51F4401F51F12100A22E51F54FC80F4431FE8
:20106B000412100812087022ED9012AC93547FF51F12100A22E5255430B40009E51F54E500
:20108B0044080210A3B42007E51F54E50210A3B4100CE51F54E54410F51F12100A22E51FB0
:2010AB0054E54402F51F12100A22BA2406201C380210DDBA25030210DDBA0F2C301C137464
:2010CB00AA120F797402120F9A7E5512086112123D22301D137455120F797405120F9A7E4A
:2010EB005512086112123D2274AA120F79742A120F9A7E5512086112123D227E0002116AB5
:20110B007E2002116A7E9002116A7E4002116A7E6002116A7EAA02116A7EA002116A7E804A
:20112B0002116A7E1002116A7EA012086112123D227EAA0211597EA002115974AA120DE8BD
:20114B00742A120E097E55120D38121246227455120DE87455120E09120D3812124622BAA8
:20116B002405201C32218EBA2502218EBA0F28301C117455120F797405120F9A120861121C
:20118B00123D22301D1174AA120F79740A120F9A12086112123D227455120F797455120F39
:2011AB009A12086112123D2212111F1210B512112912111F1210B5221211D31211E51211CB
:2011CB00F71211D31211E522751955751A55120D7B7EAA120D38121246227519AA751A2397
:2011EB00120D7B7E55120D3812124622751955751A55120D7B7E80120D38121246227519C4
:20120B0055751A55120D7B7E10120D3812124622301D012212113C12114612114122BA25E2
:20122B000302113312111F1210B512112422301DF322C2A4C2A0D2A0D2A422C284301F0708
:20124B00C280D280021256C2A0D2A0D28422C283C281D281D28322EA23F993C9A393898343
:20126B00F582E473C2873392DBD287C2873392DBD287C2873392DBD287C2873392DBD2878D
:20128B00C2873392DBD287C2873392DBD287C2873392DBD287C2873392DBD287C287D2DB45
:2012AB00223B5B9B1B021E0237022202320237022202320237023602220236021E02220260
:2012CB0022023602220222022202360222022205A520941C150222022219831B6019830231
:2012EB001E02220222218621A022ED0222022202220205198319831983196024442186191E
:20130B0083020602051E3C1E3C1E3C1E3C196022ED03060306030603120322033B035C034B
:20132B006E039F039F039F039F039F039F039F039F039F039F039F039F039F039F039F03B3
:20134B009F039F039F19831B911983039F039F039F218622362376039F039F039F05A51994
:20136B0083198319831931244421861983020605A520022002204A2002193123AC07D60733
:20138B00ED07DB07E807ED07DB07E807ED07EC07DB07EC07D607DB07DB07EC07DB15B207BF
:2013AB00DB07EC07680768061E21261C7A076807DB19831B0D19831502157207DB2186217C
:2013CB00D522FE08B308B308B3080B19831983198318B02444218619830206080B1ED11F59
:2013EB00141F741E9118EA22FE03000300029E029E029E02A802A802A802EB02A802EB03FF
:20140B00000300030002EB02A802A802A8030003000300030003000300030402A803000307
:20142B0000030003000300030002EB02A802A802A802A802A802060300030003000300033F
:20144B000021860300020602060206020602060206030002A808B508FB093F097B09BA09A2
:20146B00FD0A3E0A7D0AC00AFF0AC008B408B408B40AC00AFF0AFF0AFF0AC00AFF0AFF08FB
:20148B00B408B408B408B40AFF08B408B408B408B408B408B408B40AFF0AFF0AFF0AFF0AFE
:2014AB00FF0AFF08B408B408B408B408B408B408B408B40AFF0AFF0AFF0AFF0AFF08B40A46
:2014CB00FF00000101010202020302030001010302020203020202020202020303030001CB
:2014EB0002030202020202020303030303030302020202020203021200D0120C8B43800E4E
:20150B00782B12084B12085A1212597B0212087212101208D527EB1200D03010DD02026335
:20152B001200D0120C8BD283D284D2A0782BE6FE08120D7B121246120D381212467EFF1215
:20154B000D387D00C284C28300120D5A00D283D284DD02A16330E7EC121012D527D0120017
:20156B00D03010BF020263301C0280B4D283D284301F04D280A184D2A01200D0120C8B1224
:20158B00121B782BE6FE08120D7B121246120D38121246121012D527EB7F3C120CBA3010D1
:2015AB00CB1200D0020263D2A4D2A0D2841200D0301E2B120C8B121239782BE6FE08120EBE
:2015CB008B12123D120E2912123D121012D527EB7F14120CBA3010CF1200D00202637526F1
:2015EB000012162D50FB0E8E2712123912162D400512123D80F62526F526120E8B12123D3D
:20160B00120E2912123D121012D527E012007F7F14120CBA745512009230108B1200D002ED
:20162B000263C3309806D3E599FEC29822121073121069C2BCD284D2A4D2A01211B3121109
:20164B0015120E8BAE1C120E2912123D7F14120CBA0202637B28120872749112009222BAC5
:20166B00210302220DBA22030223E4BA35030223E4BA26030216AFBA2F03021706121073DD
:20168B00121069D284D2A4D2A012111F1210B51211107B2812087212085F12084BC2A4C2F5
:2016AB00840202EC121073121069D280D2B4D2B2D2B3D2840000C2840000D2841207591234
:2016CB00075912075912075912075912075974907E00120F78C2B2C2B400D2B4D2B2120FA7
:2016EB0078120F78120092F526EE1200922526F52612009212007F120FD92212107312100F
:20170B0069D2B4D2B2D2B3D2840000C2840000D2841207591207591207591207591207599A
:20172B00120759C019C01AC01B7400F51B74057E557FAA1205A574027EAA7F551205A57447
:20174B00057E557F901205A5D01BD01AD019120F78C2B4C2B200D2B4D2B2120759120F7885
:20176B00120092F526EE1200922526F52612009212007F120FD922BA0F0280030217B1122C
:20178B00107312106912084B121087D283D2847418120886D2A4D2A0C2A4C2A07F14120CEA
:2017AB00BAD2A0020263121073121069C2BCD284D2A4D2A01211B312110B7F14120CBA023E
:2017CB0002637F01C2A4120CBAD2A4227F01C2A0120CBAD2A0227F01C283120CBAD28322E1
:2017EB007F01C284120CBAD28422E52612009212007F221200922526F526121012221200F4
:20180B00922526F526227A083392810000000000A2A1D2A00000000000C2A0DAEB33D28179
:20182B0022120FD9120870120870121073C2A0C280121069D280120759120759C280D2A1BE
:20184B00752600C217C2127B5012087274AC12181174531218117400121811F5F0121811B2
:20186B00E5F022E51B201C07C3301201D392E3121811E51A121811E51912181122E608F522
:20188B0025851B18531BBF431B2012186E12181185181BB525012212186EE5251218117BD5
:2018AB00141208722212182C1200D0120C8B201F03120760782BC212121888201F05D2126E
:2018CB00121888121012D527ED1200D03010DC020263E608F52512186EE5251218112220A2
:2018EB001FC312182C1200D0120C8B851A28851929120760782BC2121218DDD2121218DDAA
:20190B00121012D527F0744C121811E528121811E5291218111218117B141208721200D0D8
:20192B003010C5020263C21312182CE51B121811E51E1218117400121811E51A1218117B28
:20194B00501208721200D0120FD92212186E1218111218092212182C2013CBC212121956D1
:20196B00201C08201F05D2121219561210123010EA1217F5120FD92222E5197005E51A70D3
:20198B000122851A1D85191C751A007519001210123010FAC210852D1B852D23852E1A8552
:2019AB002F1985301E85311D85321C227906543F1392A1D281C281D9F7227908D2A1D28112
:2019CB000000C28100D2810000C281A2A113D9F5F5F07906D2810000C281A2A113D9F5D20F
:2019EB00810000C2810000227908C2A1D2810000C2811392A1D2810000C281D9F57906E56E
:201A0B00F01392A1D2810000C281D9F5C2A1D2810000C281D2A12275F004E523540125F0B8
:201A2B001219B71219C50303201B03543F22540F22121069C281C2A112108712088030198E
:201A4B000B201B1074001219B7021A5F301B0574061219B722C212121A22201803B5180854
:201A6B00E5F0B52503021A75D21222121A22F52E85F02F752705752B00851A2C85192D1214
:201A8B00009A020033201B0775F019E5F0419F75F00B74089BA4FB2274021219B7E52585C8
:201AAB0018F01219F374081219B77F64DFFE740E1219B722201B047B1941C87B08121AA323
:201ACB00121A60301204DBF580A1121A90DBC92275F002E523540125F01219B7E525851854
:201AEB00F01219F3301F07E5195407B4071374081219B77B28120872121A60301203021AD6
:201B0B007622121A3C1219841200D0120C8B201803120760782B30180574FF021B2BE60833
:201B2B00F518201B0553183F613853180FE6F52508201F09121A6030120B301A05121ADB11
:201B4B006150121ABF121012D527CB1200D03010BA02026322121A3C121984752600121AA0
:201B6B00222018071200922526F526E5F01200922526F5261210123010E4E52612009212F7
:201B8B00007F120FD922121A3C301C2E74021219B7743FF5F074FF1219F374091219B77469
:201BAB00081219B77B28120872740B1219B77B281208721200D0120FD922743FF5F074FF68
:201BCB001219F37F0774061219B7DFF974021219B7743FF5F074FF1219F3201F0D740112CE
:201BEB0019B774071219B7021BFA741F1219B774081219B77B2812087274011219B77407C2
:201C0B001219B71200D0120FD922431F80121008201805C2A1021C25D2A1D2B4C280D2805D
:201C2B00752600C217C212C2D875F060121CD77400121C6930180A1200922526F526121C58
:201C4B0069C280120092D2802526F5261210123010D5E52612009212007F120FD92279084C
:201C6B003392D900D2D800C2D8A2B4D9F33322431F801210081210531210691200D0120CF4
:201C8B008B301803120760201805C2A1021C9CD2A1D2B4C280D280782B121DAA75F05012C0
:201CAB001CD7E608121C69301805E608121C69C2D900C28000D2800030B4FDD2D9121012E0
:201CCB00D527D61200D03010B5020263E51BC4540F901CE20212631CEC1D0C1D2A1D481DC3
:201CEB0075E5F07904121C6BE5193333301207448054BF021D0630170244C07906121C6B6B
:201D0B0022E5F07904121C6BE51933301206448054BFA12430170244C07907121C6B22E529
:201D2B00F07904121C6BE519301207448054BF021D4230170244C07908121C6B22E5F0E5D0
:201D4B001AA2E0E5F092E38519F0301208440853F07F021D68301705440843F0807905124A
:201D6B001C6BE5F07908121C6B22E5F0E51AA2E19215A2E09216E5F0A21592E3A21692E26B
:201D8B008519F0301207440854FB021D9D301702440C7906121C6BE5F07908121C6B2275D3
:201DAB00F040C212D217121CD7C280C217D28022D2D87908C2A10000A2D83300D2A1D9F41C
:201DCB0022C28074011220CB74001220CB000000C2A100D28000C28074051220CB121DBB5A
:201DEB00D28020E0F122C28074501220CB00C2A100D280C28074011220CB74001220CB0096
:201E0B000000C2A100D2800022C28074051220CB121DBBD28020E0F122D211120884121036
:201E2B0069C2B47F14120CBAD2D8D280D2A0D2D922121E24752600C212C280121E67121D47
:201E4B00BB1200922526F5261210123010F0D280E52612009212007F120FD922301712C285
:201E6B0017E51920E1057490021E7E74051220CB2274031220CBE51B1220CBE51A1220CB95
:201E8B00E5191220CB22121E24122179121DCC1200D0120C8B782B1221797402C28012205B
:201EAB00CB121E81E6081220CBD280C28074051220CB121DBBD280121012D527DA1200D07E
:201ECB003010CF020263121E24122179121DCC1200D0120C8B782B1221797402C2801220C2
:201EEB00CB121E81E6081220CB121012D527F5D280C28074051220CB121DBBD28020E0F114
:201F0B001200D03010CC020263121E24122179121DCC1200D0120C8B120760782B12217913
:201F2B0074ADC2801220CB121E81E13E74ADC2801220CBE6081220CB121012E6081220CBFC
:201F4B00121012D280D527E47404C2801220CBD280C28074051220CB121DBBD28020E0F122
:201F6B001200D03010AF020263121E24122179121DF11200D0120C8B782B12217974AFC23F
:201F8B00801220CB121E81E19B74AFC2801220CBE6081220CB121012D280D527EC12087047
:201FAB007404C2801220CBD280C28074051220CB121DBBD28020E0F11200D03010B702024B
:201FCB00637405C2801220CBD280227450C2801220CB00C2A100D280227401C2801220CBD9
:201FEB0074001220CB00C2A100D28022121FCC5403B4030280F622121E247F14120CBA1218
:20200B002179121DCC120870120870120870122179C28074C71220CB0000C2A10000D280A7
:20202B00120870120870120870C28074051220CB121DBBD28020E0E80205A11200DA221253
:20204B001E247F14120CBA122179121FD6121FE4121FF7122179C28074601220CB00C2A1B6
:20206B0000D280121FF7121FD6121FE4121FF7122179C28074C71220CB00C2A100D28012AA
:20208B001FF70205A11200DA22D2D8D280D2A0D2D9C2B4752600C217C21275F003C28012D6
:2020AB0020D9121DBBD2801200922526F5261210123010E6E52612009212007F120FD92220
:2020CB00790833C2A100928133D2A1D9F622E51BC4540F9020E402126320EE20F921042195
:2020EB00152116E5F01220CBE5191220CB22E5F01220CBE5191220CB22E51AA2E0E5F092C3
:20210B00E31220CBE5191220CB2222E5F01220CBE51A1220CBE5191220CB22121053121013
:20212B0069D2D8D280D2A0D2D9C2B4122179121DCC1200D0120C8B782B122179C28075F074
:20214B00021220D9E6081220CBC2A100D280C28074051220CB121DBBD2807F14120CBA1256
:20216B001012D527D41200D03010C9020263C28074061220CBC2A100D28022D2A4D285D2E1
:20218B00A0D284D2D8D280D281C2D87F1EDFFED2D830A4FD221221867EFF120E2912226C1F
:2021AB00C284120E4BD2841200922526F5261210123010E9E52612009212007F02026312ED
:2021CB0000D0120C8B782B0221DD122186121087782B12226C7E40120E29C285D285120874
:2021EB008012085AC285D2857F04DFFE30A4FD12088408121012D527D93010C31200D0027B
:20220B00026312107312106912218612226C7E90120E29C28500D285C284120E4BD28412C7
:20222B00009212009212007F02026312107312106912218612108712226C7E20120E29C29A
:20224B008500D28512226C1208807ED0120E29C28500D2857F08DFFE30A4FD12088402054E
:20226B00A1E519A2E09293A2E19292A2E29291A2E39290A2E492B2A2E59286A2E69297A25C
:20228B00E792DAE51AA2E092B4A2E192D9A2E292A1C2A0E51AA2E39293A2E49292A2E592A6
:2022AB0091A2E69290A2E792B2E51BA2E09286A2E19297A2E292DAA2E392B4C392D992A1A9
:2022CB00D2A022D2A4D285D2A0D284D281C2D8D2D87FFFDFFE7FFFDFFEC2D87F0ADFFED2AB
:2022EB00D8221222CE0221A31200D0120C8B782B02230C1210731210691222CE121087786F
:20230B002B12235A12226C12085AC28500D2857F03C28400000000120E4BD2845480F5F004
:20232B00E65480B5F01008121012D527D43010B81200D0020263DFD9F52E85F02F752705B6
:20234B00851B2B851A2C85192D12009A020263C019C01AC01B7EAA12241E7E5512242A7E43
:20236B00A012241ED01BD01AD019221210731210691222CEC019C01AC01B7EAA12241E7ED4
:20238B005512242A7E8012241E7EAA12241E7E5512242A7E1012241ED01BD01AD0190205D5
:2023AB00A11210731210691222CEC019C01AC01B7EAA12241E7E5512242A7E8012241E7E42
:2023CB00AA12241E7E5512242A7E30D01BD01AD019913630A4FD0205A112107312106912E3
:2023EB0022CEC019C01AC01B7EAA12241E7E5512242A7E9012241ED01BD01AD01912226CE5
:20240B00C284120E4BD28412009212009212007F020263751955751A55751B0091362275B5
:19242B0019AA751A2A751B0091362212226C120E29C285000000D28522FA
:00000001FF
